:100000000EC026C025C024C023C022C021C020C0ED
:100010001FC01EC01DC01CC01BC01AC019C01124A7
:100020001FBECFEDCDBF10E0A0E6B0E0ECE1F1E007
:1000300003C0C89531960D92A036B107D1F710E0F4
:10004000A0E6B0E001C01D92A036B107E1F701C003
:10005000D7CF86E187BB81E088BB00000000B09B62
:1000600029C020E047E1EEE1F0E031E048BB8E2F0F
:100070009F2F0197F1F738BB8E2F9F2F0197F1F734
:100080002F5F203199F78CE898E30197F1F720E092
:1000900047E1EEE1F0E031E048BB8E2F9F2F019762
:1000A000F1F738BB8E2F9F2F0197F1F72F5F20318B
:1000B00049F1F2CF20E047E1EEE1F0E031E048BB6A
:1000C0008E2F9F2F0197F1F738BB8E2F9F2F01970F
:1000D000F1F72F5F203199F78AE599E20197F1F75F
:1000E00020E047E1EEE1F0E031E048BB8E2F9F2FAA
:1000F0000197F1F738BB8E2F9F2F0197F1F72F5FF4
:10010000203199F785B7877E806185BF85B780628A
:0C01100085BF889585B78F7D85BF089559
:00000001FF
